:020000040000FA
:020000006E2868
:0800080045288C0081018316DC
:100010000313C030810508008C008101831603138F
:10002000C030810501308104831203130B110B1DB5
:1000300017288C0B162808009900051208308C0030
:100040002D2019180516191C0512990C2D208C0B42
:10005000212805162D202D2008000C308D00332876
:1000600001308D0033288D0B332808009A01642855
:100070001011950303193F2802301C2091019301B0
:100080009401950112081C2008008B138B1B452836
:100090009C00030E9D0083010A089E008A018313C1
:1000A00004089F000B1C6528861B5C28101C642814
:1000B00010109014910A6428101864281014101558
:1000C0009201901C920A90100B101F0884001E08C9
:1000D0008A001D0E83009C0E1C0E0900831603135C
:1000E00081010512831203130516910192019301F8
:1000F000940195018B018B158B17832849300520BE
:1001000002301320901001309307031C8A289407B3
:0E0110000318950A90187E28101938208328AD
:02400E00F13F80
:00000001FF
